:100000006F28A0008417800484138E010C1C8E00BE
:10001000102003196A28102003196A2810206A2862
:1000200020088E0601308C008D01000820050E0688
:10003000031D08008C0A03198D0F152808008F0175
:100040008E00FF308E07031C8F07031C6A280330C5
:100050008D00DF302D2021288D01E83E8C008D0998
:10006000FC30031C36288C07031833288C076400E7
:100070008D0F33280C183C288C1C40280000402889
:1000800008008E000330442894000F080D02031D61
:100090004B280E080C0204300318013003190230FB
:1000A0001405031DFF306A28103094008D018C0167
:1000B000930C920C031C62280E088C070F0803187F
:1000C0000F0F8D078D0C8C0C910C900C940B5828F5
:1000D00010086A2883130313831264000800831630
:1000E000083085008601831285018601D1290130FF
:1000F0008C0005308400083001200C08A6000D0893
:10010000A70026088C0027088D008F015030412061
:10011000031D8C28A901080026088C0027088D00E3
:100120008F0175304120031D98280130A900080077
:1001300026088C0027088D008F018E304120031D7A
:10014000A4280230A900080026088C0027088D008A
:100150008F01A2304120031DB0280330A900080000
:1001600026088C0027088D008F01BB304120031D1D
:10017000BC280430A90008000530A90008000511BA
:10018000831605118312303086003C301F20051580
:1001900083160511831286013C301F20051183163A
:1001A00005118312303086003C301F200515831660
:1001B0000511831286013C301F200511831605119D
:1001C000831286013C301F2005158316051183120A
:1001D00086013C301F200511831605118312C030A3
:1001E00086003C301F2005118316051183120F3045
:1001F00086003C301F200511831605118312C03084
:1002000086003C301F2005118316051183120F3024
:1002100086003C301F2005118316051183128601CC
:100220003C301F2005118316051183120F30860004
:100230003C301F20051183160511831230308600D3
:100240003C301F20051583160511831286013C30B2
:100250001F200511831605118312303086003C30B3
:100260001F20051583160511831286013C301F20BF
:10027000051183160511831286013C301F200515D8
:1002800083160511831286013C301F200511831649
:1002900005118312C03086003C301F2005118316E3
:1002A000051183120F3086003C301F200511831684
:1002B00005118312C03086003C301F2005118316C3
:1002C000051183120F3086003C301F200511831664
:1002D0000511831286013C301F200511831605117C
:1002E00083120F3086003C301F2005118316051144
:1002F0008312303086003C301F200515831605110F
:10030000831286013C301F200511831605118312CC
:10031000303086003C301F200515831605118312EE
:1003200086013C301F2005118316051183128601BA
:100330003C301F20051583160511831286013C30C1
:100340001F200511831605118312C03086003C3032
:100350001F2005118316051183120F3086003C30D3
:100360001F200511831605118312C03086003C3012
:100370001F2005118316051183120F3086003C30B3
:100380001F20051183160511831286013C301F20A2
:1003900005118316051183120F3086003C301F2093
:1003A000FD29850186010515831605118312033089
:1003B0008F00E830202005118316051183120130CB
:1003C000A400A5010130A800640009302802031828
:1003D000FC29240886002408920025089300023096
:1003E0008E008F015420A4001108A50003308F0057
:1003F000E8302020A80FE4298601BF2829088D00B5
:10040000053C031C1B2A8D0D0B228C000D100B22AA
:100410008A000C08820002308A000D08820700342E
:10042000BF340034BF340034BF3402341C340034D1
:10043000BF340034BF34FD2905158316051183121E
:0A0440000F308600FD296300232A17
:02400E00FD3F74
:00000001FF
